:1000000012C0189518951895189518951895189563
:100010001895189518951895189518951895189578
:100020001895189518958FE58DBFC0E4E8E34E2E1E
:1000300084E08EBFD4E0F4E05F2EEEEFF3E0A0E6C4
:10004000B0E0A89584B7082E877F84BF88E1992700
:1000500081BD91BD88278D933197E9F783E389B9F5
:1000600080E080BD88E18AB9662483E886B980ECA7
:1000700087B9B99ABA9ABB9ABC9A379A07B1007FE6
:10008000006007B9AED0A0E6B0E08D939C93A0E6E7
:10009000B0E00D911C910C3B52E015070CF401C02F
:1000A00002C080E088BBA0E6B0E00D911C910C3B43
:1000B00052E0150780E014F009F081E08F93A0E68C
:1000C000B0E00D911C910E3E52E0150780E00CF45B
:1000D00081E09F918923882309F402C082E088BBD4
:1000E000A0E6B0E00D911C910E3E52E0150780E0B5
:1000F00014F009F081E08F93A0E6B0E00D911C911F
:10010000003253E0150780E00CF481E09F918923D1
:10011000882309F402C086E088BBA0E6B0E00D9118
:100120001C91023553E0150780E014F009F081E0DE
:100130008F93A0E6B0E00D911C91043853E01507B1
:1001400080E00CF481E09F918923882309F402C0A8
:100150008EE088BBA0E6B0E00D911C91043853E01E
:10016000150714F009F001C002C08EE188BBA0E2BF
:10017000B4E0E0E6F0E054D007D00ED0E1E0F0E0EB
:1001800012D07BCFF894FFCFA0E2B4E08D9188230A
:1001900011F005D0FBCF08958DE001D08AE05D9B82
:1001A000FECF8CB9089588EE93E00CD03197D9F743
:1001B00008953197F1F70895689462F80895E894E6
:1001C00062F80895EF93FF93EE27E82BE92B31F0C7
:1001D000EAEFF0E03197F1F70197D1F7FF91EF9156
:1001E0000895369A3699FECF369A3699FECF84B165
:1001F00095B10895000F111F221F331F0895009518
:100200001095209530950F5F1F4F2F4F3F4F08954A
:10021000019110810EC001911191219130810BC08B
:100220000191108117FF05C03FEF2FEF04C000813F
:1002300011272227332737FF03C0E1DF8DE28D939B
:10024000CF93DF93CF92DF92EF92AA24BB24CC24EA
:10025000DD24EE2440E2CAE0DD2755E093E3888107
:10026000890F87FD9F7083FD907F891B89935A9525
:10027000A9F7C0DFAA1CBB1CCC1CDD1CEE1C4A95D8
:1002800051F7E894EFE0FF2782910ED0EB30E0F7D2
:100290001EF068948A2D0CD088278D93EF90DF9004
:1002A000CF90DF91CF910895982F829501D0892F1B
:1002B0008F70805D26F0803309F4089568948D93E3
:0202C00008959F
:00000001FF
